:100000000C9492050C94BA050C94BA050C94BA059C
:100010000C94BA050C94BA050C94BA050C94BA0564
:100020000C94BA050C94BA050C94C7160C943617A8
:100030000C94BA050C94BA050C94BA050C94BA0544
:100040000C94BA050C942A1A0C94BA050C94BA05AF
:100050000C94BA050C94BA050C94BA050C94681962
:100060000C94BA050C94BA050C94BA050C94BA0514
:100070000C94BA050C94BA050C94BA050C94BA0504
:100080000C94B2190C94BA050C94BA050C94BA05E8
:100090000C94BA050C94BA050C94BA050C94BA05E4
:1000A0000C94BA050C94BA050C94BA059C59000C32
:1000B0009C48000C9C450018D49C35000C9C4500C5
:1000C00010E280F0FFFF07FF077707FF077707FFC2
:1000D000077707FF077707FFFF07070707070707E8
:1000E00007070707070707070707070707079C5BB7
:1000F00000089C4A00089C47000CD39C3B000A9CCB
:100100003E000FE280F0FFFF475717FF077707FF1A
:10011000077707FF077707FFFF07070707070707A7
:100120000707070707070707070707079C60000877
:100130009C4C00089C43000CD29C3C000A9C48004C
:100140000FE280F0FFFFFF07FF077707FF07770742
:10015000FF077707FFFFFF070707070707070707DF
:1001600007070707070707070707944B0010943F87
:100170000018945200109466001880F0F844561746
:10018000FF87B7076E0CF80001030707070707038F
:10019000010094510018944100109460001880F000
:1001A0007C82FFC3DB83B7867C0000010101010173
:1001B0000000944F0012943E000C945F001280F0F7
:1001C0007CA2AB8BFF87B7867C0000010101010197
:1001D0000000903D0014904F001E80F07CFE83FFD5
:1001E00087B787FE7C0000010101010100009042F9
:1001F000000C9053001080F01C3E5155453E1C9061
:10020000470008904C000C80F01C3E7F417F3E1C54
:100210000000000000700100C0000C00CAA77C0AAA
:10022000CAE22D0A534248195EF55112003000000F
:100230000027450040941C0014F3190504F1110433
:1002400020040000044110040004000010420801D2
:100250005E14450F40F001005955551351555D0D81
:100260008C927C085755550D5E55550D51520C0119
:100270005E55550F5655550F00A0000000A4000014
:1002800000C2280080A228008062080040500D00B3
:100290005E7455079C92241F5F555D0D9C1445119B
:1002A0005F1425075F5555115F5114015E54551DAC
:1002B0001F41101F40F44500100421071F41181D65
:1002C0001F0441105EF0041F9C10041F5E54450F74
:1002D0005F9214035ED4451F5F92341B5655550D33
:1002E00041F005011F0421071F4208011FE4410FCF
:1002F0001743181D07C1090151564D1100F0450063
:1003000000F0010040F4010080100C0010044110C6
:10031000050115012501370149015D0172018801BF
:100320009F01B801D201EE010B022A024B026E02BC
:100330009302BA02E40210033E037003A403DC0339
:10034000160454049604DC0426057505C805200629
:100350007D06E0064807B7072D08A9082D09B90949
:100360004D0AEA0A900B400CFA0CC00D910E6F0F6B
:100370005A1053115A1272139A14D3152017801859
:10038000F519801B221DDE1EB420A622B524E4260A
:100390003429A72B402E0031080809090A0B0B0C41
:1003A0000D0E0E0F10111213141617181A1B1D1F05
:1003B00020222427292B2E3134373A3D4145494EFE
:1003C00052575C62686E747B838A939BA5AEB9C4F6
:1003D000CFDCE9F7000102030406080C00F4F8FA88
:1003E000FCFDFEFF90480064904A0064904C00645D
:1003F000904D0064904F00C880F04241434B205420
:100400004F205449544C45004245434F4D452050E0
:10041000454E4E494C45535300434F4E54494E555B
:1004200045002435205155414452494C4C494F4ECA
:100430002100594F5527564520474F540000808EC4
:1004400015F555554E5555F5158E80000364949756
:100450006A35555555356A9794640380404E95F535
:1004600055554E5555F5158E8000016292936A35AB
:10047000555555352A7794946300809C2AEAAAAA98
:100480009CAAAAEA2A9C8000639494635D6AAAAA43
:10049000AA6A5D6394946300808E15F555554E5598
:1004A00055F5954E4080639494772A3555555535CA
:1004B0006A9392620100000000000000000007073C
:1004C00009020100FF015D0707F8010500EE01A820
:1004D0000909DC010A00D201DE0909C0013200B2BB
:1004E00001820909A00164009201870B0B7C01F4D1
:1004F000016A01A5130B4401E8032C0159130B06F3
:10050000018813EE0076150BC4001027AC00C20F53
:10051000100000000000000043414E43454C004FD6
:100520004B00903700789036008C903500A09034C6
:1005300000B4903300C8903200DC903100F090306D
:1005400000FF80F0464F52202341524455424F59FC
:10055000204D454D45204A414D004F424E2D5931C9
:10056000362056455220302E303100C0C6CFDFFF36
:10057000FB73037CFEFFC7E3FF7F3E00FFFFFF1B13
:100580001B1B03000303FFFFFF0303000000000029
:10059000000000808080800000000000000000005B
:1005A00000000080E0F058AC56AB55AB5500FF01A1
:1005B00001010202040810608000003FFFAA55AA52
:1005C00055AA55AA55A85FAC5CAC5CAC5CAC5C0CA5
:1005D000CF3C0000000103060D1A152A252A252A02
:1005E0002522151209040201000000FFFF57AB5736
:1005F000AB57AB57AB03FF808080000000000000CA
:10060000000000FFFF55AA55AA55AA55AA00FF00F1
:100610000000010102040830C000001F7FD5AA5568
:10062000AA55AA55AA54AF56AE56AE56AE562E8609
:10063000671E000000000103060D0A1512151215B1
:1006400012110A090402010000000000000000006D
:10065000008080C0C0C0C08080800000000000001A
:10066000000000C0F078AC56AB55AA55AA00FF00B8
:100670000000010102040830C00000FFFF55AA5528
:10068000AA55AA55AA00FFFEAE56AE56AE56AE56B5
:1006900007FE001F171512151215121512101F173D
:1006A0001215121512151215101F000000A040A0FF
:1006B0000028104438827C007C8ED6DADA827C00F6
:1006C000383800387CFE00FC09E00C630CD710675A
:1006D0001390104352454449540047414D4520531F
:1006E0005441525400492057414E54202435205142
:1006F00055414452494C4C494F4E0000004445433B
:10070000454D42455220323032330050524F47520D
:10071000414D4D4544204259204F424F4E4F00001D
:10072000544849532050524F4752414D204953009D
:1007300052454C454153454420554E444552005482
:100740004845204D4954204C4943454E53452E00C1
:100750001B00000000000080C4663B391E0F02FE33
:10076000FC6009CDF6FFFFFF3E463E5E2FC7F7FA5D
:10077000FC7F9F6F170B0403000000000000C0E027
:10078000F8FC7F9F6F170B05050400000080E7FF52
:10079000FFFFFC00F0000080F8FEFF7FBF5F2F131B
:1007A0000D020180E0F8FFFF7F1FC3F1FD7FBFCF87
:1007B0006270BC5F4F07FBFF7FBF5300FCFFFFFF72
:1007C000FFE1EEE1E0F0F070B0B8582C160278FFCF
:1007D000FFFFFF7C9D661A05020000060EBCBFBF2E
:1007E0005F2F170986E1E0F0F767AB4C03000000CC
:1007F00000000000030B0B0B0505050505050200B5
:100800000201010000000105020100000001030BCC
:100810000B0B0B05050502020100000000000000A3
:1008200001050502010000000000000000000000BA
:10083000000000000001030B0502010000000000A1
:1008400000000000000000000000806018060202A6
:1008500082828282828282424242BEC03810080472
:10086000048242C1010101020206FC80C06010083E
:1008700004048242C101010102020CF080C0201078
:100880000804048242C101010102020CF00060A0D0
:1008900010080402120E070181E1790D0701010120
:1008A0000905834C50A0C0C0781E030101C121A1DD
:1008B0006101010101C121A16101010101C131CD2C
:1008C000330C000000304C4340404060A061000009
:1008D00000000001FEE13F07010000C030CCF23D06
:1008E0000E0300008060F81F07010000806098E69A
:1008F000390E0300008070F81F07010000C030CCE3
:10090000F23D0E030000C030ECFB1C07848405029E
:10091000030180E0701E07018060C0828141A2B5A2
:10092000CAF1791E070100C040404744434140409E
:1009300040C00704030100806098661906010000AA
:10094000007FC1818181818384834140A0A05028A0
:10095000140B3F40808080808083824140A05028DB
:10096000140B043F41808080808083824140A050EE
:1009700028140B047FC0808080808083824140A047
:100980005028140B0C7782834241A1505028147BCD
:10099000C78180808082834140A050EDF39C878195
:1009A0008080609C631C030101E19F83834343417A
:1009B00040A05028160906010000000000000000B9
:1009C0000002020202020202010100000000000017
:1009D0000000000202020202020101000000000009
:1009E00000000000020202020202030100000000F7
:1009F00000000000020282E2F27A72313100D8F087
:100A0000F06080F0FA727101808000000080D2F204
:100A1000F2E2E2628201010000000202020202C26E
:100A2000E1C0C0C00000000002028281010101009B
:100A300000000000000080C0C0E0E0C0C0D5F08D24
:100A400014A1C881CFD9F1AF20000000000024001C
:100A500027002A002D00300000000000250028009B
:100A60002B002E00310004080201104080401020AD
:100A70004080408008020401804020100201108064
:100A80001020404020040404040403040502020270
:100A90000204030202020206060606060604040217
:100AA000020204041C0A130AB50F090A6411B109F1
:100AB0004B0EDD136E12080B000202020000090447
:100AC00000000102020000052400100105240101BC
:100AD0000104240206052406000107058103100015
:100AE0004009040100020A0000000705020240005C
:100AF00000070583024000000403090412010002FC
:100B0000EF020140412336800001010203014172DE
:100B10006475696E6F204C4C430041726475626F5E
:100B20007900061B11241FBECFEFDAE0DEBFCDBF78
:100B300011E0A0E0B1E0E4EBFFE302C005900D920C
:100B4000AC33B107D9F726E0ACE3B1E001C01D92A8
:100B5000A93DB207E1F715E0C2E9D5E004C021974D
:100B6000FE010E94D21FC139D107C9F70E94231B81
:100B70000C94D81F0C940000E3E8F2E080E0A0E0C1
:100B8000B8E000800EBC8111012C1197A0FDFDCFB3
:100B90000192B9F70DB40895CF93DF93DC0177FF8D
:100BA00013C022273327261B370B842F042E000C5B
:100BB000990B281739072CF4460F70E060E01416E3
:100BC00044F0DF91CF9108951416DCF7603471057D
:100BD000C4F7A038B105A8F7262FCB01840F911DCB
:100BE00047FD9A958134910514F040E4461B277027
:100BF0009FEF022E01C0990F0A94EAF7420F621B81
:100C0000710977FF02C0695F7F4F83E07595679533
:100C10008A95E1F7FB01F695FE2FEE27F795E7950C
:100C2000EA0FFB1FED57FD4F28E030E06FEF70E05B
:100C300014163CF6483064F4D901A41BB10947FDF1
:100C4000B395EB0102C0D595C795AA95E2F79C2311
:100C50008081982B90834850E058FF4F9FEFE8CF5A
:100C60006F927F928F929F92AF92BF92CF92DF92BC
:100C7000EF92FF920F931F93CF93DF9330E0F90130
:100C8000E80FF91F1E161F060CF09EC08038910554
:100C90000CF09AC0FB01E00FF11D1E161F060CF0B0
:100CA00093C0603471050CF08FC0DB0177FF04C086
:100CB000AA27BB27A61BB70BA770BB27FB0177FD95
:100CC0003796C3E0F595E795CA95E1F777FF07C03A
:100CD000319768E070E0EB01CA1BDB0BDE01A02E50
:100CE000A694A694A694B12C077019F0DFEFAD1A64
:100CF000BD0ABF018A01EF01D695DC2FCC27D7951D
:100D0000C795C80FD91FCD57DD4FAE0EBF1E48E0A7
:100D100050E04A018A1A9B0AA616B70609F454C085
:100D20006830710509F450C06F3FEFEF7E070CF497
:100D300041C050E040E07E01F0E8EF0EF11C4217A8
:100D40005307C4F5FC01E40FF51FE038F10594F5F5
:100D5000F7FD2DC06F3F7607A1F1FA01E00FF11FFB
:100D6000E4916E01C40ED51EF0E03F010A2E01C0D1
:100D7000660C0A94EAF7F601708067286082109783
:100D8000B1F06730710599F0FA01E00FF11FE491BD
:100D90006701C40ED51EF0E03F01082C02C0759417
:100DA00067940A94E2F7F6017080672860824F5FCB
:100DB0005F4FC5CF6F5F7F4F020F131FC058DF4FCC
:100DC000ABCF109709F7F3CFDF91CF911F910F9120
:100DD000FF90EF90DF90CF90BF90AF909F908F905B
:100DE0007F906F900895FC0180916A02882311F131
:100DF0003FB7F89482E08093E9002091F200822FBF
:100E000090E01816190614F481E090E0882339F078
:100E1000289844E6409369024091F10040832223E0
:100E200039F02091F200211103C02BE62093E80055
:100E30003FBF08958FEF9FEF08952FB7F89483E099
:100E40008093E9009091E800892F807295FF04C09B
:100E50009091F20080E4891B2FBF08958091610278
:100E600081110DC082E080935D0284E080935E0278
:100E70001092600210925F0281E0809361028DE522
:100E800092E00895CF93DF931F92CDB7DEB76983C9
:100E9000DC01ED91FC910280F381E02D41E050E016
:100EA000BE016F5F7F4F09950F90DF91CF9108953D
:100EB00083E08093E9008091F200882319F08AE3AF
:100EC0008093E80008950E941D0790E00895CF9355
:100ED000DF931F92CDB7DEB7FC018485958597FD22
:100EE00008C02FEF3FEF358724870F90DF91CF9118
:100EF0000895CE0101960E94F306019719F48981A5
:100F000090E0F3CF8FEF9FEFF0CF0F931F93CF932E
:100F1000DF931F92CDB7DEB78C01FC0184859585E8
:100F200097FF0BC0CE0101960E94F306019771F462
:100F3000898190E0F80195878487F80184859585FB
:100F40000F90DF91CF911F910F9108958FEF9FEF39
:100F5000F1CFFC018485958597FD0BC09FB7F89470
:100F600082E08093E9008091F2009FBF90E00196BB
:100F700008959FB7F89482E08093E9008091F20091
:100F80009FBF90E0089540915702509158022091E0
:100F900055023091560242175307B4F49091E8007D
:100FA0009570E1F39091E80092FD19C08093F100F3
:100FB000809157029091580201968F739927892B3F
:100FC00019F48EEF8093E8008091570290915802B7
:100FD0000196909358028093570281E0089580E033
:100FE0000895DF92EF92FF920F931F93CF93DF93B9
:100FF000D82E8A01EB017B01E40EF51ECE15DF052C
:1010000059F0D7FE12C0FE0184910E94C3072196B9
:101010008111F4CF0FEF1FEFC801DF91CF911F9126
:101020000F91FF90EF90DF9008958881EECF0F939E
:101030001F93CF93DF931F92CDB7DEB782E08983F2
:1010400042E450E066EB7AE080E80E94F1070E94FB
:101050002E07DC0112960D911C910115110589F0E6
:10106000D801ED91FC910280F381E02DBE016F5F0C
:101070007F4FC801099597FD04C0F80100851185CF
:10108000ECCF89810F90DF91CF911F910F9108953F
:10109000615030F02091F100FC0120830196F8CFDF
:1010A000289884E680936902089580913A02089511
:1010B000AF92BF92CF92DF92EF92FF920F931F9366
:1010C000CF93DF936C017B018B01040F151FEB01A4
:1010D0005E01AE18BF08C017D10759F06991D6015B
:1010E000ED91FC910190F081E02DC6010995892BCD
:1010F00079F7C501DF91CF911F910F91FF90EF908C
:10110000DF90CF90BF90AF9008953FB7F894809153
:10111000300290913102A0913202B091330226B593
:10112000A89B05C02F3F19F00196A11DB11D3FBF1F
:10113000BA2FA92F982F8827BC01CD01620F711DEE
:10114000811D911D42E0660F771F881F991F4A95E8
:10115000D1F708958F929F92AF92BF92CF92DF9274
:10116000EF92FF926B017C010E9485084B015C01AC
:10117000C114D104E104F104B9F00E948508681992
:1011800079098A099B09683E73408105910580F3BE
:1011900021E0C21AD108E108F10888EE880E83E048
:1011A000981EA11CB11CE4CFFF90EF90DF90CF9070
:1011B000BF90AF909F908F9008958F929F92AF9223
:1011C000BF92CF92DF92EF92FF920F931F93CF9334
:1011D000DF936C017B018A0180910D01882309F462
:1011E0005CC080916A02882309F457C080915C0238
:1011F00080FF05C08091E00082608093E000E801FC
:10120000B12C8AEFA82E93E0892E2AE3922E209704
:1012100011F4BB20D9F10E941D0781110AC0AA94C4
:10122000AA20D9F161E070E080E090E00E94AA0875
:10123000EECF8C171D0611F00CF08C2F9FB7F89491
:101240008092E9002091E80025FD02C09FBFDFCF1A
:10125000282F30E0C21BD30BF701815020F04191C1
:101260004093F100FACFE20EF31EBB2021F09092E2
:10127000E800B12CEBCF8091E80085FDE7CF90929C
:10128000E800BB24B394209709F3F3CF5D9884E67C
:1012900080935B02101611063CF081E090E0F601AD
:1012A0009383828310E000E0C801DF91CF911F910A
:1012B0000F91FF90EF90DF90CF90BF90AF909F90F5
:1012C0008F900895BC0190E080E00C94AA088FB143
:1012D0008095807F669B88601C9B84600895109237
:1012E0003A023E983F9808953E9A3F9A81E0809353
:1012F0003A02089580E0E3E8F2E081118FEF0024E4
:1013000081938193819381930394D1F710922E025C
:1013100010922D0210922C0210922B020895EF923F
:10132000FF920F93CF93DF937C01EB0100E22EE756
:1013300045E458E00E943006BE01605E7F4F04E144
:1013400021E542E557E0C7018F960E943006DF9104
:10135000CF910F91FF90EF90089583E08093270243
:101360000895E0912702E33059F0F0E0EE0FFF1FFF
:10137000E353F94F85919491FC01099510922A024B
:1013800008959C0190911F0293306CF484E09802C0
:10139000F0011124ED5EFD4F33832283718360835E
:1013A0009F5F90931F02089510921F026DEA79E0EB
:1013B0008AED96E00E94C1096AE57CE083ED96E043
:1013C0000E94C1091092200281E0809329029CE1D1
:1013D0009093260295E39093250298E4909324023B
:1013E0009BE090932302109222028093210280932B
:1013F000270280932A0208958091280281508093C9
:101400002802811102C00E94D40981E080932A023F
:10141000089580912702811104C08EE180932802F3
:1014200008950C94D4099091280291509093280229
:1014300081E0911180E0089588E780932802089563
:10144000FF920F931F93CF93DF93EC01FB018081F9
:101450009181A881B9812B8139E0F32E2F9D9001D4
:101460001124F901EB54FB4FE4918C010A1B1B0B77
:10147000F0E031964E0F5F1F0417150754F5FB017E
:1014800043814F9DA0011124FA01EB54FB4FE491DD
:10149000A81BB90BEA171B06E4F0F901EA54FB4F4D
:1014A000A591B491FB01228130E08A8190E0B901DD
:1014B000681B790BA617170664F0FA01EA54FB4F74
:1014C00045915491BC01621B730B81E046171706CE
:1014D0000CF480E0DF91CF911F910F91FF90089560
:1014E0008F929F92AF92BF92EF92FF920F931F93B2
:1014F000CF93DF938C01AB01DC01ED90FC90119751
:10150000F194E194F1081396EC91B9E0EB9FF001AE
:101510001124EB54FB4FE491CE2FD0E0EC16FD06E6
:101520009CF1F801238139E0239FF0011124E75455
:10153000FB4F4591549180913D0290913E02A091C4
:101540003F02B0914002840F951FA11DB11D409133
:1015500041025091420260914302709144024A015B
:101560005B01EFEF8E1A9E0AAE0ABE0A8115F1EEFC
:101570009F07F5EFAF07F5E0BF07B8F0915EA54F05
:10158000B540B501A401EBCF6EE072E00E94200AE5
:101590008111C7CFDF91CF911F910F91FF90EF90F5
:1015A000BF90AF909F908F90089580933D0290934D
:1015B0003E02A0933F02B0934002411531EE530723
:1015C00035EF630735E07307A8F440934102509369
:1015D0004202609343027093440281E080933B0295
:1015E000EC16FD0614F420930D02D80113961C92FC
:1015F00081E0D0CF8FEF90EEA5EFB5E08093410270
:1016000090934202A0934302B093440280933D0220
:1016100090933E02A0933F02B0934002DECFEDE3F1
:10162000F2E02081318145E0429FC001439F900D4F
:1016300011244281538167E0649F9001659F300DC2
:101640001124820F931F875C9A474481558169E07A
:10165000649F9001659F300D1124280F391F46812A
:1016600057816BE0649FC001659F900D1124820F2C
:10167000931F408551856DE0649F9001659F300DFB
:101680001124820F931F0895CF92DF92EF92FF9261
:101690000F931F93CF93DF93082F142F469FE001E2
:1016A000479FD00D1124F12CE12C60E074E284EF0F
:1016B00090E0A7019E010E943B1F21503109410982
:1016C000510991E02115310581E0480751056CF081
:1016D00060E970ED83E090E0A7019E010E943B1F4E
:1016E000215031094109510993E0013059F003308B
:1016F000F9F0DF91CF911F910F91FF90EF90DF9064
:10170000CF90089510933E0180918100887F892BAE
:101710008093810030938900209388001092850087
:101720001092840080916F00826080936F00E1CFFF
:1017300010933F01D0933D01C0933C0180919100F3
:10174000887F892B80939100309399002093980093
:1017500010929500109294008091710082608093A5
:101760007100C7CF811116C010927C028091720265
:1017700081110AC080913702E0913802F09139025C
:10178000908180958923808342E064EF71E083E05B
:101790000C94440B80917702811110C080916F00EE
:1017A0008D7F80936F0080913402E0913502F0913B
:1017B0003602908180958923808308950895FF9251
:1017C0000F931F93CF93DF93EC01909182029923A3
:1017D00009F464C08B01913071F4809181028823F7
:1017E00051F0809180028F3F09F058C080E00E9444
:1017F000B20B10928102E0917E02F0917F02099576
:10180000FF24F3948F2580937D0230E020E0A9012E
:101810009801220F331F441F551FDE010E945A1FDB
:101820006C507E4F8F4F9F4F28EE33E040E050E0EA
:101830000E946D1F809182028130A1F480937C020E
:10184000209378023093790240937A0250937B027E
:1018500083E042E0BE01DF91CF911F910F91FF9095
:101860000C94440BF092770220937302309374022D
:10187000409375025093760280918102882351F043
:1018800081E0909180029F3F09F080E08093720296
:1018900081E0DFCF8FEF80938002FACFDF91CF918D
:1018A0001F910F91FF90089564E170E08BE492E046
:1018B0000C94DF0B0E94540C82E08093270281E09D
:1018C00080932A0208958091D70690E080959095A4
:1018D0002091D8062C7030E082239323892B39F095
:1018E0000E94540C81E08093270280932A0208957D
:1018F000E0915302EE2359F14091200220911F0202
:10190000022E000C330B0E2E000CFF0BCF01840FA8
:10191000911D47FD9A95820F931FB9010E94AA1F3E
:10192000482FDC01AA0FBB1FAA0FBB1FAD5EBD4F26
:101930006D917C91672B51F3809320026AE070E0F7
:1019400088EB91E00E94DF0B81E080932902809177
:1019500021028823C1F08091D806887090E0209100
:10196000D70630E02095309582239323892B59F0B8
:1019700080913A02811120C00E9474090E94540C87
:1019800081E0809329028091D806847090E02091B4
:10199000D70630E02095309582239323892B79F068
:1019A000E091200284E0E802F0011124ED5EFD4F99
:1019B0000190F081E02D09940E946F09DFCF089516
:1019C0000C94780C0E94540C82E0809312020895CB
:1019D0000E94540C1092120281E080932A02089512
:1019E000CF93DF93C091200286E0C802E00111246A
:1019F00069960E94540C10921F026CEA76E18FE106
:101A000095E00E94C10968EE7CE088E195E00E94C3
:101A1000C10988E280932602C09325028FE2809359
:101A200024028BE08093230281E080932202809342
:101A300021028093200280932902DF91CF910895A3
:101A4000FF920F931F93CF93DF9301E010E0FF24E9
:101A5000F394E0916E02F0916F02AF014F5F5F4F20
:101A600050936F0240936E022491822F807FC22F89
:101A7000CF70D22FD370803821F48D2F0E94B20BFB
:101A8000E8CF803909F03FC0E0917E02F0917F02FB
:101A900009958F2580937D02E0916E02F0916F028F
:101AA000CF01019690936F0280936E02E491809132
:101AB0006D0290918202D91760F6D13021F4909195
:101AC00077029111C6CF8E0F87FDC3CFE82FF0E0CC
:101AD0008C3390F4E856FC4FE4916E2F70E081E077
:101AE000D11103C0F0927C0283E04C2F46954695BD
:101AF0004E5F0E94440BADCFEE0FFF1FE856FD4F27
:101B000065917491ECCF87FD3FC03296F0936F02E0
:101B1000E0936E02FA014491A0913C01B0913D0125
:101B2000322F242F0E948F1F6C507E4F8F4F9F4F5C
:101B300028EE33E040E050E00E946D1F20937802D1
:101B40003093790240937A0250937B02809178021D
:101B500090917902A0917A02B0917B02892B8A2B15
:101B60008B2B61F481E090E0A0E0B0E080937802FC
:101B700090937902A0937A02B0937B02DF91CF9188
:101B80001F910F91FF900895803DA1F4F093710291
:101B9000E093700280916B02882309F45ACFEC2FF6
:101BA000F0E0EC52FC4FE491C0916D02EC0FE09339
:101BB0006D024FCF803E21F5C11109C080917002A6
:101BC0009091710290936F0280936E0242CF809148
:101BD0006B028F5F80936B02980102C0220F331F4C
:101BE000CA95E2F7821713064CF3509371024093A3
:101BF000700280916C0280936D0210926B0229CF6B
:101C0000803F09F026CF10928102B8CF0F931F9327
:101C1000CF93DF938C01D62F80918102882349F1E5
:101C200080918002861790F1C0E080918202C817EF
:101C300028F48C2F0E94B20BCF5FF7CF1092810255
:101C4000D0938002109371020093700210936F0280
:101C500000936E0210926D0210926C0210926B0251
:101C600081E080938102DF91CF911F910F910C94BD
:101C7000200D80917702882319F381E090918002F2
:101C8000961708F080E080937202DACFDF91CF914F
:101C90001F910F91089560E084EE93E00E94060E7C
:101CA000809145029091460201969093460280935E
:101CB000450281E080933B02EDE4F1E0138234962B
:101CC00082E0ED30F807D1F71092400188E090E013
:101CD00090930F0280930E028BE1809310028AE0B2
:101CE000809311021092280210924A011092490129
:101CF00010924C0110924B0110924101109212026D
:101D000081E080932A020895EF920F93CF93DF939F
:101D100077FF0CC088279927861B970B2817190671
:101D200009F00CF47CC0260F70E060E057FF0FC094
:101D3000EE27FF27E41BF50B802F002E000C990BDC
:101D4000E817F9070CF06BC0040F50E040E02223C5
:101D500009F465C0603871050CF061C010160CF014
:101D60005EC0403451050CF05AC0CB01820F911D6A
:101D70008138910514F020E8261B942FFA01E00F1A
:101D8000F11D07FDFA95E134F10514F000E4041BA0
:101D900097708FEF092E01C0880F0A94EAF7090F98
:101DA000491B510957FF02C0495F5F4F93E05595AA
:101DB00047959A95E1F75695542F4427579547959F
:101DC000640F751F6D577D4F48E050E0AFEFB0E0F6
:101DD00010162CF5083064F4FA01E01BF10907FD38
:101DE000F395ED0102C0D595C795EA95E2F78C23EE
:101DF000E1100DC08095FB01922F30813823319383
:101E00009150D9F7085060587F4F8FEFE1CFFB0119
:101E1000922F3081382B31939150D9F7F3CFDF9146
:101E2000CF910F91EF900895BF92CF92DF92EF92F2
:101E3000FF920F931F93CF93DF936A30C9F4809181
:101E40002D0290912E02069690932E0280932D02E1
:101E500010922C0210922B0281E090E0DF91CF9142
:101E60001F910F91FF90EF90DF90CF90BF9008955A
:101E700080EE860F803480F740912B0250912C0227
:101E80009A01CA0105968538910560F5C0912D0229
:101E9000D0912E02CE0106968634910518F5109148
:101EA000000184E0689FF0011124E057FE4FC590C7
:101EB000D590E590F490F0E000E170E060E0C0FCC7
:101EC00018C0B12C111116C0F694E794D794C7949A
:101ED0006F5F7F4F6630710591F72F5F3F4FFF5F58
:101EE000F63059F74A5F5F4F50932C0240932B0214
:101EF000B3CFB12E2038310538F7CB018C0F9D1FA1
:101F00008034910508F7E1E081FDE4E080FDEE0F0B
:101F100082FDE295887F089FD0011124A20FAD5762
:101F2000BD4F8C91B0FE03C08E2B8C93CDCFE0952E
:101F30008E23FBCF0F931F93CF93DF938C01D0E0C1
:101F4000C0E0F801EC0FFD1F6491662341F083EDC2
:101F500096E00E94140F892B11F02196F2CFCE014A
:101F6000DF91CF911F910F9108958F929F92AF9221
:101F7000BF92CF92DF92EF92FF920F93CF93DF93B6
:101F8000809128028F50990B63E070E00E94AA1F95
:101F90008AE39AEAA3EEBEEE04C0B695A79597959C
:101FA00087956A95D2F7C82FC1708FE7C89F802D9B
:101FB000112493E894BD9FEF97BD91EF909380001B
:101FC0008093880010928A000E947A09209128024A
:101FD00088E790E0821B91096CE270E00E94AA1FE2
:101FE0004B018BE8C82E85E0D82E9CE1A92EB12CA0
:101FF000F12CE12CD0E081E090E08E149F0411F0F0
:1020000090E080E08C9FB0018D9F700D9C9F700DC3
:102010001124645F7F4F00E228E1A601C5010E9400
:1020200030068FEFE81AF80A88E1A80EB11C80E6A6
:10203000C80ED11C83E0E816F104E9F608E020E2BE
:102040004BE655E06CE270E084E490E00E943006DC
:1020500080E190E090932C0280932B028AE390E041
:1020600090932E0280932D028AE595E00E949A0FAC
:1020700081E090E090932C0280932B0210922E022C
:1020800010922D0284E495E0DF91CF910F91FF90A3
:10209000EF90DF90CF90BF90AF909F908F900C9477
:1020A0009A0F089590E080E0089597FF0DC02227D1
:1020B0003327281B390B4217130629F024F0480F49
:1020C00090E080E031F408954423E9F380389105ED
:1020D000D4F760347105B8F79C01240F311D213805
:1020E000310514F040E8481B362F377021E001C05D
:1020F000220F3A95EAF7FB0133E0F595E7953A951B
:10210000E1F7F695FE2FEE27F795E795E80FF91F13
:10211000ED57FD4F8081822B81934150D9F7D3CF6A
:10212000CF92DF92EF92FF920F931F93CF93DF93A3
:1021300080912A02882391F10E947A090BE010E035
:10214000C5EED6E0FE0184918B3141F165E170E08E
:10215000CE010E94E71E7C016C01DD24282F3DEF9B
:102160003203C0011124805C9F4F90932C02809316
:102170002B0210932E0200932D02CE010E949A0F83
:102180008FEFC81AD80ACC0DDD1D86E090E0E11073
:1021900002C082E090E0080F191FD4CFDF91CF91E9
:1021A0001F910F91FF90EF90DF90CF9008954F9285
:1021B0005F926F927F928F929F92AF92BF92CF92D7
:1021C000DF92EF92FF92CF93DF93CDB7DEB72C97DC
:1021D0000FB6F894DEBF0FBECDBF0E947A09809083
:1021E0002802912C6627772768197909CB01770F88
:1021F000AA0BBB0B89839A83AB83BC839FEF891A9D
:10220000990A092C000CAA08BB0889819A81AB8124
:10221000BC81881A990AAA0ABB0A0E94861E6D838D
:102220007E838F839887C0902802D12C4424552424
:102230004C185D08052C000C660877089FEFC91A3A
:10224000D90A0D2C000CEE08FF08C418D508E608C2
:10225000F7080E94861E69877A878B879C876D8125
:102260007E818F819885A50194010E943B1F898002
:102270009A80AB80BC80860E971EA81EB91E698509
:102280007A858B859C85A70196010E943B1FDC0106
:10229000CB01840D951DA61DB71DB4012C960FB65C
:1022A000F894DEBF0FBECDBFDF91CF91FF90EF90CE
:1022B000DF90CF90BF90AF909F908F907F906F9066
:1022C0005F904F900C948F09CF92DF92EF92FF9224
:1022D000E0912702F0E0EE0FFF1FE953F94F8591DF
:1022E0009491FC0109950E942A1E6C01990FEE0839
:1022F000FF080E948508C616D706E806F90631F0E1
:102300006C257D258E259F250E94D51E8091270254
:10231000833031F081E0FF90EF90DF90CF9008950F
:1023200082E0F9CF6F927F929F92AF92BF92CF924D
:10233000DF92EF92FF920F931F93CF93DF93A090C2
:10234000230222E0922E9A0C10912402F090250292
:102350006F2C0F2C000C7708630181E0C81AD1089C
:10236000C09126020C2E000CDD0B22E0210FBE01D5
:1023700061507109E12C092DA60183ED96E00E94C0
:10238000840E80912202882331F194E0B92EB10E9F
:10239000E2E06E1A710822974B2DB301CE010E9424
:1023A000551084E08A0DB301680F711D87FD7A9581
:1023B000615071094B2DCE010E945510492DB60177
:1023C000CE010E94CC05CE018B0D911D492DB60189
:1023D00001970E94CC05D0E0C0E083E1C82E82E0E6
:1023E000D82E80911F02082E000C990BC817D90710
:1023F0000CF04AC0F60182819381009709F441C034
:10240000AF2C0F2C000CBB0820912602022E000CD2
:10241000330B245F3F4F40912002042E000C550BDC
:10242000C417D50759F544E050E0241B350B309311
:102430002C0220932B02B0922E02A0922D020E9419
:102440009A0F80912002082E000C990BC817D9070B
:1024500071F460912602062E000C770BEE24E394B3
:1024600005E025E0A50183ED96E00E94840EF6E0EC
:10247000FF0E219684E0C80ED11CB3CF50E040E09F
:10248000D4CFF394F394F5CF809121028823B1F057
:1024900040E150E067EB76E08DE696E00E94DE1EBC
:1024A00060913A02E6E06E9FB00111246555794FC4
:1024B00046E050E08DE796E00E94DE1E1092290271
:1024C000DF91CF911F910F91FF90EF90DF90CF9010
:1024D000BF90AF909F907F906F900895BF92CF92E2
:1024E000DF92EF92FF920F931F93CF93DF93809130
:1024F0001202823009F4D6C08111DEC00E947A092E
:10250000CDE4D1E019E08B818823C1F0819FC00127
:102510001124FC01EA54FB4FA591B491FC01EB544A
:10252000FB4F2491FC01E954FB4F459154916A8182
:1025300070E00A2F888199810E943006249622E05B
:10254000CD30D20701F74091280246954695437059
:102550008EE1489FA0011124435C5B4F6091100203
:1025600070E000E12FE080910E0290910F020E9436
:10257000300660913D0270913E0280913F02909141
:102580004002CAE72AE0C22ED12CE12CF12C2C2FDC
:1025900030E030932C0220932B0210922E021092E6
:1025A0002D02A70196010E946D1FB22E032F142F3A
:1025B000D52F605D83ED96E00E94140F6B2D702F78
:1025C000812F9D2FC650CA3441F460914102709111
:1025D0004202809143029091440261157105810588
:1025E0009105A9F600914102109142022091430207
:1025F00030914402012B022B032B11F0CB3438F61F
:10260000D0E0D0932C02C0932B0210922E02109295
:102610002D0264E283ED96E00E94140F8091410246
:1026200090914202A0914302B09144028038904FB1
:10263000AA4FB240A8F1EE24E3940FE020E848E16D
:1026400050E070E060E083ED96E00E94840E80919F
:10265000280284FF25C01092000182E290E090934E
:102660002C0280932B028AE190E090932E028093BB
:102670002D0282E394E00E949A0F83E190E0909310
:102680002C0280932B0280E290E090932E028093A4
:102690002D0282E294E00E949A0F81E08093000173
:1026A00010922A02DF91CF911F910F91FF90EF902E
:1026B000DF90CF90BF90089580912902811104C0CE
:1026C00080912A02882361F30E949211E9CFCF936F
:1026D000C0912A02CC2341F00E947A0970E060E0A8
:1026E00090E080E00E948F0980912902811102C050
:1026F000CC2319F0CF910C949211CF910895CF93E0
:10270000DF9380913C02813009F054C080E692E072
:102710009093480280934702F999FECF4FE452E428
:102720006EE476E180E692E00E942E1F80914702DF
:102730009091480204969093480280934702F99939
:10274000FECF60914702709148024AE050E08DE36D
:1027500092E00E94161FC0914702D09148022A962B
:10276000D0934802C09347020E940F0BF999FECF05
:10277000BC01CE010E94361F809147029091480211
:1027800002969093480280934702C0913A0282E0F9
:1027900090E00E94021FC81729F06C2F82E090E0A1
:1027A0000E94201F82E080933C0210923B02DF9146
:1027B000CF91089584E692E0BECF2F923F924F9240
:1027C0005F926F927F928F929F92AF92BF92CF92C1
:1027D000DF92EF92FF920F931F93CF93DF9300D07E
:1027E00000D000D01F92CDB7DEB72091120281E059
:1027F000223009F458C22111ACC22091D80626FB20
:10280000882780F990E025FB662760F970E0861B39
:10281000970B60910E0270910F02860F971F8237FF
:10282000910514F081E790E097FF02C090E080E00E
:1028300090930F0280930E0224FB442740F950E04E
:10284000822F022E000C990B8827990F881F992739
:10285000481B590B80911002840F813308F080E3EC
:10286000863008F486E080931002809128028F5F02
:102870008093280222FF30C280914B0190914C013D
:10288000803A29EF920728F4019690934C018093A7
:102890004B01C0904B01D0904C0100914901109127
:1028A0004A010C0D1D1D005A1F4F10934A01009341
:1028B0004901612F77277F836E8310920D028DE08F
:1028C000A82E82E0B82E9DE4E92E91E0F92ED701E2
:1028D00013968C911397882369F08D919C91119791
:1028E000EE81FF818E1B9F0B8D939C93BF01C701CF
:1028F0000E94700AF4E0EF0EF11CAE14BF0439F729
:102900002E813F812115310509F4C5C0922F8827FA
:10291000081B190B10934A01009349018D2D8695D0
:102920008F5F8B3008F4DDC1982F843108F093E17C
:102930009A509B838A3008F089E02E803F80882E51
:10294000912C6FEF861A960A092C000CAA08BB0876
:1029500080914001A82FB0E0BD83AC83AA0FBB1FBC
:10296000AA0FBB1FBA83A983FD01E35BFE4F8381DE
:10297000811184C0BB81CB2ED12CF12CE12CC81449
:10298000D904EA04FB049CF4240135014C185D08C9
:102990006E087F0841F00E94861EA30192010E94EA
:1029A0003B1F2B013C01C40CD51CE61CF71C098104
:1029B0001A81035B1E4FF801C3820E94861E28E025
:1029C00030E040E050E00E943B1F20E830E0221958
:1029D0003309C901860F971FD80111969C938E93D6
:1029E0001396EC91B9E0EB9FF0011124EA54FB4FF0
:1029F0008591949101E410E0081B110946E050E034
:102A000060E070E007301105A4F00E94861E012EE0
:102A1000000C220B330BA901980126503109410902
:102A200051090E943B1FAB01BC014A5F5F4F6F4FD2
:102A30007F4F8C819D81880F991F880F991FFC0102
:102A4000E35BFE4F7F01E981FA81E35BFE4F428346
:102A5000B101C7010E94700A811110C02E813F810F
:102A6000203231050CF44DC18091400190E0C196B7
:102A700060E370E00E94AA1F80934001EE81FF8115
:102A800084E090E0B0970CF439C1281A390A121486
:102A900013040CF45DCFE0910D02EE2359F029E010
:102AA000E29FF0011124E554FB4F8591949162E07F
:102AB0000E94060EE0910D02EE2309F443C139E0B5
:102AC000E39FF0011124E354FB4F25913491822FB1
:102AD00064E20E949E1F8093440136E0822F632FA0
:102AE0000E949E1F292F0E949E1F909343012093B6
:102AF000420188E08093410180914101209142018F
:102B0000829F202D112490914301899F902D1124A3
:102B100030914401839F802D112433E834BD90957A
:102B200097BD91EF909380002093880080938A0056
:102B30008091D806887090E02091D70630E02095EB
:102B4000309582239323892B09F43EC00E94540CB4
:102B500010921F0268EE7CE089E194E00E94C109B6
:102B600060EF7CE088E094E00E94C10962EE7CE0C6
:102B70008AEF93E00E94C1098AE08093260287E1F0
:102B8000809325028BE68093240281E180932302C7
:102B900081E0809322028093210210922002809390
:102BA000290280913B0281110E947F1383E884BD3A
:102BB0008FEF87BD81EF8093800010928800109284
:102BC0008A0081E0809312028091D70690E0809580
:102BD00090956091D806A62FB0E0A823B923BA83B8
:102BE000A9832091450130914601409147015091C0
:102BF000480182E0C82ED12CE12CF12C812C912CA3
:102C000054018394412C64EA562E6AE9662E63E0EF
:102C1000762ED501C4010C2C04C0880F991FAA1F61
:102C2000BB1F0A94D2F7E981FA818E239F23892B57
:102C300091F0A6E0B0E00E945A1FA30192010E9409
:102C40006D1FA70196012250310941095109260F34
:102C5000371F481F591FFFEFCF1ADF0AEF0AFF0A7D
:102C600068E0C616D104E104F10499F62093450109
:102C7000309346014093470150934801293F3C4619
:102C80004B48534061F48FE790EFAAEFB2E0809396
:102C9000410290934202A0934302B093440281E028
:102CA00080932A0282E027960FB6F894DEBF0FBE0B
:102CB000CDBFDF91CF911F910F91FF90EF90DF90EB
:102CC000CF90BF90AF909F908F907F906F905F90CC
:102CD0004F903F902F90089510924C0110924B010D
:102CE000D8CD31E03B8326CE34E0C30ED11C8823FF
:102CF00071F0E981FA81E35BFE4F138281E090E09D
:102D0000C4CE7DE4C72E71E0D72E10E000E08091A4
:102D1000400180171106A1F0D60113968C918823EB
:102D200079F050E040E0B701C6010E94200A0F5F31
:102D30001F4F00331105C1F6882309F495CED9CF72
:102D400080E0F5CF80914101882309F4D5CE8150F0
:102D5000D1CE0E94780CA6CFCF9361E082E295E0BD
:102D60000E94060EEDE3F2E01482158216821782AD
:102D70001082118212821382C1E0C0933B020E9432
:102D80007F1310921202C0932A02CF9108951F92CE
:102D90000F920FB60F9211248F939F938091E100B1
:102DA0009091E100937F9093E10083FF0FC0109218
:102DB000E90091E09093EB001092EC0092E3909385
:102DC000ED0010926A0298E09093F00082FF22C01A
:102DD00093E09093E9009091F200992319F09AE31F
:102DE0009093E80090915B02992341F090915B02EF
:102DF000915090935B02911101C05D9A909169028C
:102E0000992341F090916902915090936902911138
:102E100001C0289A84FF18C08091E2008E7E8160F4
:102E20008093E2008091E1008F7E8093E1008091A9
:102E30005C028E7E806180935C029F918F910F90E7
:102E40000FBE0F901F90189580FFF7CF8091E20082
:102E50008E7E80618093E2008091E1008E7E80937F
:102E6000E10080915C028E7E8160E5CF1F920F921F
:102E70000FB60F921124CF92DF92EF92FF920F9331
:102E80001F932F933F934F935F936F937F938F93F2
:102E90009F93AF93BF93EF93FF93CF93DF93CDB700
:102EA000DEB76C97DEBFCDBF1092E9008091E800DD
:102EB00083FF25C068E0CE0145960E94480882EF56
:102EC0008093E8008D8987FF39C09091E80090FFDA
:102ED000FCCF982F907609F034C19E894F89588D88
:102EE0002F89F88C911131C0803861F580915A0298
:102EF0008093F1001092F1008EEF8093E8006C96C1
:102F00000FB6F894DEBF0FBECDBFDF91CF91FF911A
:102F1000EF91BF91AF919F918F917F916F915F9151
:102F20004F913F912F911F910F91FF90EF90DF9064
:102F3000CF900F900FBE0F901F9018959EEF90931B
:102F4000E800C7CF1092F100D5CF913059F481112C
:102F5000D3CF4130510581F680915A028D7F809305
:102F60005A02CACF933049F48111C6CF413051057E
:102F700019F680915A028260F2CF953041F4809127
:102F8000E80080FFFCCF20682093E300B5CF9630A7
:102F900009F0A9C00B8D1C8D22E01092E90010925F
:102FA000580210925702F2122EC01092560210923E
:102FB00055020E9417081F8299E09983FA8291E0D6
:102FC0009E8390EA98879AEF9987209157023091D3
:102FD0005802275F3F4F3C832B838D831092E9007B
:102FE0001092580210925702109356020093550205
:102FF00049E050E0BE016F5F7F4F80E00E94F10723
:103000000E94170879CF10935602009355020E9430
:103010002E07DC0112960D911C910115110509F482
:1030200051C1D801ED91FC910480F581E02DBE01E4
:103030006B5E7F4FC8010995009709F03EC1F8010A
:1030400000851185EACFF3E0FF120EC08F89882337
:1030500009F440C0823061F440E867E08AE19BE017
:103060000E94D31A811148CF81E28093EB0047CFB1
:10307000813029F440E86BE08EE09BE0F1CF8330B3
:1030800099F70E942E07DC011296ED90FC908E01BC
:103090000F5F1F4F6801E114F10479F0D701ED9142
:1030A000FC910680F781E02DB801C7010995080F52
:1030B000111DF701E084F184EECFD8011C92F601D6
:1030C00001900020E9F73197BF016C197D0940E0BC
:1030D000C601C6CF68EF7AE0FB01449150E080E87A
:1030E0000E94F10709CF973009F4BECF983021F440
:1030F00081E08093F10000CF993009F0FDCE83701C
:1031000009F0B2CFE7E1F1E081E031E096E321910F
:10311000222371F08093E9003093EB00DF011197D7
:103120002C912093EC009093ED008F5F873079F71E
:103130008EE78093EA001092EA008F8980936A02FA
:10314000DBCE8B8D9C8D1092E9001092580210926C
:1031500057029093560280935502898D811192C037
:103160008E899D89913A49F4813209F07DCF47E0FB
:1031700050E066E071E080E0B3CF913209F074CFA7
:10318000833269F48F89988DB0E0A0E080930201CA
:1031900090930301A0930401B0930501ADCE80325A
:1031A00069F48091E80082FFFCCF67E086E091E05F
:1031B0000E9448088BEF8093E8009ECE823209F08F
:1031C0009BCE8F8980930D01EEEFFFE7859194915F
:1031D0008B3F9C4D51F1E0E0F8E080910601909129
:1031E0000701A0910801B0910901803B9440A1051D
:1031F000B105F1F480910D0180FD1AC0EE3F8AE027
:10320000F80789F587E797E79183808380916000CD
:103210008093590288E19BE00FB6F894A8958093BB
:1032200060000FBE9093600067CEEEEFFAE0D5CF5E
:10323000808191818737974709F05ECEA89580916C
:1032400060008861809360008091590280936000E3
:10325000EE3F2AE0F20789F08091FE0A9091FF0A82
:103260009183808349CE808191818737980751F27D
:103270009093FF0A8093FE0AC5CF1092FF0A109226
:10328000FE0A3ACE0E942E07DC0112960D911C9187
:103290000115110509F4E8CED801ED91FC910190DA
:1032A000F081E02DBE016B5E7F4FC8010995811151
:1032B00023CEF80100851185EBCF181619060CF402
:1032C0001BCED2CEF1E0FF12BECE6CEF7AE004CF7F
:1032D0001F920F920FB60F9211242F933F938F934B
:1032E0009F93AF93BF938091490290914A02A0911E
:1032F0004B02B0914C0230912F0223E0230F2D3767
:1033000058F50196A11DB11D20932F02809349020B
:1033100090934A02A0934B02B0934C0280913002EA
:1033200090913102A0913202B09133020196A11D19
:10333000B11D8093300290933102A0933202B0937A
:103340003302BF91AF919F918F913F912F910F9039
:103350000FBE0F901F90189526E8230F0296A11D0F
:10336000B11DD2CF1F920F920FB60F9211242F933F
:103370003F934F935F936F937F938F939F93AF93FD
:10338000BF93EF93FF9380917C02882329F1809172
:103390007202811121C080917D0281111DC0609156
:1033A00078027091790280917A0290917B0220914B
:1033B0003F0130E050E040E00E946D1F6230710537
:1033C0008105910548F490913702E0913802F0911F
:1033D00039028081892780838091780290917902D7
:1033E000A0917A02B0917B02892B8A2B8B2BE9F07A
:1033F0008091780290917902A0917A02B0917B023B
:103400000197A109B1098093780290937902A09362
:103410007A02B0937B02892B8A2B8B2B31F480911B
:103420008102882399F00E94200DFF91EF91BF91B6
:10343000AF919F918F917F916F915F914F913F914C
:103440002F910F900FBE0F901F90189580E00E9453
:10345000B20BEBCF1F920F920FB60F9211242F9346
:103460003F934F935F936F937F938F939F93AF930C
:10347000BF93EF93FF9380917702882309F472C082
:103480008091730290917402A0917502B0917602BE
:10349000892B8A2B8B2B09F451C080917D028111DD
:1034A0001DC06091730270917402809175029091B9
:1034B000760220913E0130E050E040E00E946D1F16
:1034C000623071058105910548F490913402E091D4
:1034D0003502F091360280818927808380917302C2
:1034E00090917402A0917502B0917602892B8A2B7B
:1034F0008B2B99F08091730290917402A0917502C8
:10350000B09176020197A109B1098093730290935B
:103510007402A0937502B0937602FF91EF91BF9170
:10352000AF919F918F917F916F915F914F913F915B
:103530002F910F900FBE0F901F901895109272024E
:103540001092770280916F008D7F80936F00809141
:103550003402E0913502F091360290818095892302
:103560008083DBCF80917D028111D7CF6091730280
:1035700070917402809175029091760220913E01C3
:1035800030E050E040E00E946D1F6230710581051F
:10359000910518F690913402E0913502F0913602CF
:1035A00080818927DDCFEF92FF920F931F93CF93F6
:1035B000DF93F82E192FE62E042F81E0860F880F57
:1035C0000E94C30783E00E94C307CF2DD12FEC0ECA
:1035D000FD2EF11CCE15DF05B9F007FF13C0FE016B
:1035E00084910E94C307182F80E00E94C3078123A3
:1035F00021968111EFCFDF91CF911F910F91FF9015
:10360000EF9008958881EDCF81E0F5CFE3E8F6E013
:103610001382128288EE93E0A0E0B0E08483958369
:10362000A683B78381E291E0918380838FEF9FEF40
:1036300095878487E3EDF6E01382128283E391E0BD
:10364000918380830895789484B5826084BD84B525
:10365000816084BD85B5826085BD85B5816085BD8D
:1036600080916E00816080936E0010928100809145
:1036700081008260809381008091810081608093CD
:103680008100809180008160809380008091910012
:10369000826080939100809191008160809391007D
:1036A000809190008160809390008091C10084603F
:1036B0008093C1008091C10082608093C10080919D
:1036C000C10081608093C1008091C30081608093BC
:1036D000C3008091C00082608093C0008091C200CE
:1036E00081608093C20080917A00846080937A0028
:1036F00080917A00826080937A0080917A00816064
:1037000080937A0080917A00806880937A0010928A
:103710006A0210925A0210925C028091D700816076
:103720008093D70080EA8093D80089B5806189BDF5
:1037300089B5826089BD09B400FEFDCF61E070E00B
:1037400080E090E00E94AA088091D8008F7C806180
:103750008093D8008091E000807F8093E00080918A
:10376000E1008E7E8093E1008DE08093E200559A27
:10377000209A81EC80937C0085B1806F85B984B1FB
:10378000877E84B984B1876E84B95E9A5F988AB166
:10379000806D8AB9769A6E9881B3806F81BB899863
:1037A00080B38D7080BB80E58CBD81E08DBD85E0F0
:1037B00090E00E9462095F9A85E090E00E946209B1
:1037C0005E985C98EDE3FAE08AE49AE024912EBDDD
:1037D00000000DB407FEFDCF31968E179F07B1F79D
:1037E0005C9A81E880936400809165008160809399
:1037F00065000E94BC050E94670987FF15C05C98A0
:1038000085EA8EBD00000DB407FEFDCF5C9A2E98B0
:103810002F982D988091640080628093640081E0ED
:1038200083BF889513BEFCCF0E94670982FF46C004
:103830002D980E94670984788438D9F42D9A88ECF1
:1038400090E00E9462092F9882E090E00E94021F9F
:103850008F3F29F06FEF82E090E00E94201F84EFFD
:1038600091E00E9462092F9A0E9467098478843847
:10387000D9F30E94670984718431D9F42D9A88ECB8
:1038800090E00E9462092E9882E090E00E94021F60
:10389000882329F060E082E090E00E94201F84EFFE
:1038A00091E00E9462092E9A0E9467098471843116
:1038B000D9F388EC90E00E946209B6CF2D9A82E09D
:1038C00090E00E94021F882369F10E94740980E140
:1038D0008093010185E598E090937F0280937E02BA
:1038E000809182028823C9F190E023E080918202D6
:1038F000981768F5911119C0809171008D7F8093A0
:10390000710080913702E0913802F09139023081E4
:103910008095832380838091650088608093650013
:103920009F5FE4CF0E946F09D2CF80916F008D7F9F
:1039300080936F0080913402E0913502F09136025D
:10394000308180958323808320938100E9CF10927A
:103950007202109277021092810281E080938202BB
:10396000EAE8FAE08491EBE6FAE0249190E0880F2F
:10397000991FFC01E85AF54F45915491FC01E65B13
:10398000F54FA591B4918C91822B8C938091650019
:10399000877F809365001092900089E0809391006A
:1039A00050933902409338022093370280E00E94FE
:1039B000B20B80E692E09093480280934702F99917
:1039C000FECF80E692E00E940A1F24E632E03093A8
:1039D0004802209347026F3472448E44964109F0A6
:1039E0005EC0F999FECF4AE050E064E672E08DE3F4
:1039F00092E00E94F21EC0914702D09148022A969E
:103A0000D0934802C0934702F999FECFCE010E949D
:103A1000101F8C012296D0934802C09347020E9447
:103A20000F0B8017910709F03AC082E080933C02A7
:103A300010923B0280913A02882309F43DC00E9413
:103A40007409E0915402B6E0EB9FF0011124EC55AB
:103A5000F54F85919491FC010995EE24E394D6E00D
:103A600000E010E0DD24D394FF24FA948FE0C82E08
:103A70008FB7F8944091490250914A0260914B02ED
:103A800070914C028FBF80914F028823C1F0109239
:103A90004F020115110561F30E940000E9CFEDE32B
:103AA000F2E08AE0DF011D928A95E9F781E08093D8
:103AB0003C0280933B02BECF0E946F09C2CF80912F
:103AC0005002F42FF81B8F2F90910101F91738F451
:103AD0008F5F8917F0F6E3BE889513BEDACFD092D8
:103AE0004F024093500280914D0290914E020196F8
:103AF00090934E0280934D028091D8068093D70612
:103B00000E9467098093D8061092530210925202C5
:103B1000982F907F09F44FC0909151029F5F94318C
:103B20000CF046C09093510290915102913011F0E7
:103B30009F30A1F485FDF092520286FF05C090915E
:103B400052029F5F9093520287FDF092530284FFCE
:103B500005C0809153028F5F80935302E09154021D
:103B6000DE9FF0011124EA55F54F85919491FC01F7
:103B70000995C82FE0915402DE9FF0011124E85509
:103B8000F54F85919491FC0109950E94BC058091A7
:103B90005402C81709F47DCFC0935402DC9FF00192
:103BA0001124EC55F54F85919491FC01099571CF45
:103BB000C0925102B9CF10925102D0CF8F929F92F2
:103BC000AF92BF92CF92DF92EF92FF92CF93DF93AB
:103BD000EC01688179818A819B816115710581057C
:103BE000910521F464E279ED8BE597E02DE133EF67
:103BF00041E050E00E943B1F49015A019B01AC018A
:103C0000A7EAB1E40E945A1F6B017C01ACEEB4EF4D
:103C1000A50194010E94681FDC01CB018C0D9D1D44
:103C2000AE1DBF1DB7FF03C00197A109B04888832F
:103C30009983AA83BB839F77DF91CF91FF90EF9009
:103C4000DF90CF90BF90AF909F908F9008950E948B
:103C5000DE1D08958EE091E00E94DE1D0895B0E023
:103C6000A0E080930E0190930F01A0931001B093F8
:103C7000110108958F929F92AF92BF92CF92DF92DF
:103C8000EF92FF92CF93DF93EC01688179818A8173
:103C90009B81611571058105910521F464E279ED3F
:103CA0008BE597E02DE133EF41E050E00E943B1FB0
:103CB00049015A019B01AC01A7EAB1E40E945A1FD5
:103CC0006B017C01ACEEB4EFA50194010E94681F6A
:103CD000C60ED71EE81EF91EF7FE06C081E0C81A00
:103CE000D108E10880E8F80AC882D982EA82FB821A
:103CF000C701B6019F77DF91CF91FF90EF90DF90E2
:103D0000CF90BF90AF909F908F9008958F929F9289
:103D1000AF92BF92CF92DF92EF92FF926091120129
:103D20007091130180911401909115016115710535
:103D30008105910521F464E279ED8BE597E02DE1B1
:103D400033EF41E050E00E943B1F49015A019B01C3
:103D5000AC01A7EAB1E40E945A1F6B017C01ACEEF2
:103D6000B4EFA50194010E94681FC60ED71EE81E7D
:103D7000F91EF7FE06C081E0C81AD108E10880E804
:103D8000F80AC0921201D0921301E0921401F0924D
:103D90001501C701B6019F77FF90EF90DF90CF909C
:103DA000BF90AF909F908F90089560931201709391
:103DB000130180931401909315010895FB01DC0118
:103DC00002C005900D9241505040D8F70895FC0173
:103DD0000590615070400110D8F7809590958E0F36
:103DE0009F1F0895DC01CB01FC01F999FECF06C0AD
:103DF000F2BDE1BDF89A319600B40D9241505040A9
:103E0000B8F70895F999FECF92BD81BDF89A992728
:103E100080B50895A6E1B0E044E050E00C94F41EB3
:103E2000A8E1B0E042E050E00C94F41EDC01CB01CC
:103E300003C02D910E94211F41505040D0F708959A
:103E4000262FF999FECF1FBA92BD81BD20BD0FB6B6
:103E5000F894FA9AF99A0FBE01960895242F0E94B9
:103E6000211F252F0E94211F0C94361F0E94201F06
:103E7000272F0C94211F052E97FB1EF400940E94FF
:103E8000521F57FD07D00E946D1F07FC03D04EF450
:103E90000C94521F50954095309521953F4F4F4FB0
:103EA0005F4F089590958095709561957F4F8F4FE6
:103EB0009F4F08950E948F1FA59F900DB49F900D56
:103EC000A49F800D911D11240895B7FF0C945A1FD3
:103ED0000E945A1F821B930B0895A1E21A2EAA1B5F
:103EE000BB1BFD010DC0AA1FBB1FEE1FFF1FA217AA
:103EF000B307E407F50720F0A21BB30BE40BF50BA7
:103F0000661F771F881F991F1A9469F7609570952F
:103F1000809590959B01AC01BD01CF010895A29FB2
:103F2000B001B39FC001A39F700D811D1124911D8D
:103F3000B29F700D811D1124911D0895991B79E088
:103F400004C0991F961708F0961B881F7A95C9F729
:103F50008095089597FB072E16F4009407D077FDFF
:103F600009D00E94BE1F07FC05D03EF490958195B4
:103F70009F4F0895709561957F4F0895AA1BBB1BB5
:103F800051E107C0AA1FBB1FA617B70710F0A61B59
:103F9000B70B881F991F5A95A9F780959095BC017A
:103FA000CD010895EE0FFF1F0590F491E02D0994C7
:043FB000F894FFCFB3
:103FB4000110FFFFFFFF00E100000000000001000E
:103FC40000000100000000C180810000000000002A
:103FD400004207DD0863075807A90767078507003C
:0C3FE400000000140F580852105110008B
:00000001FF
